:040000006F00A020CD
:100004000000000000000000481600004A1600002E
:1000140000000000080200000000000000000000D2
:1000240008020000080200000000000000000000B8
:1000340008020000000000000802000000000000A8
:10004400080200000802000008020000000000008E
:1000540008020000AA1700000802000008020000BD
:100064000802000008020000080200000802000064
:1000740008020000601600000802000008020000E8
:100084000802000008020000080200000802000044
:100094000802000008020000080200000802000034
:1000A4000802000008020000080200000802000024
:1000B4000802000008020000080200000802000014
:1000C4000802000008020000080200000802000004
:1000D40008020000080200000802000000000000FE
:1000E400000000000000000000000000000000000C
:0C00F40000000000000000000000000000
:10010000397101436EC619A0397141536AC866CA74
:1001100062CC5ECE19A0397101535AD056D252D456
:100120004ED64AD826DA22DC06DE330161408282CE
:1001300041114AC026C222C406C68282B24D410184
:10014000024D924C224CB24B4101024B924A224A40
:10015000B2494101024992442244B24041018280A5
:100160003D432A876373C3029377F700BDEFADE584
:10017000937606FF3D8ABA960CC34CC30CC74CC796
:100180004107E36BD7FE11E28280B306C3408A06C3
:100190009702000096966780A6002307B700A30683
:1001A000B7002306B700A305B7002305B700A304D3
:1001B000B7002304B700A303B7002303B700A302CB
:1001C000B7002302B700A301B7002301B700A300C3
:1001D000B7002300B700828093F5F50F9396850052
:1001E000D58D93960501D58D61B79396270097021B
:1001F000000096968682E78086FA9680C1171D8F4A
:100200003E96E374C3F8A5B701A09701002093813F
:100210006160175100201301E1DE1715000013057E
:100220002571970500209385E5DD1706002013064C
:10023000E63263FAC5008322050023A055001105AC
:100240009105E3EAC5FE138581D4938501016377A7
:10025000B500232005001105E36DB5FEFD42739046
:1002600002BC8D42739042809302800873900230EA
:1002700097020000938242D993E232007390523089
:10028000EF10805E971200009382223E739012342A
:1002900073002030B727014093870740631DF500A6
:1002A000EFF21FE98545130500201D238145130545
:1002B0000020392B45B582805C413707F1E01307F8
:1002C000F7EF944D7D8F9C41D58FD44DD58FD44180
:1002D000A206D58FD98F5CC11C4537F7F1FF1307F4
:1002E000D77FD4457D8F9C49D58F94458606D58F81
:1002F000D98F1CC55C55370710FF7D177D8FDC2912
:10030000FD1793F7F70FD207D98F5CD582801C4574
:1003100089C593E717001CC58280F99BEDBF5C413E
:1003200093F5F50F01C6DD8D4CC1828093C5F5FFB5
:10033000FD8DDDBF1C4591C537075000D98F1CC509
:1003400082803707B0FF7D17F98FD5BFA54763F7C8
:10035000B7048D47138765FF3307F7020328C500ED
:100360009D47B397E70093C7F7FFB3F70701B3962D
:10037000E600DD8E54C5994763E3C70495477D16B3
:100380003306F6025859FD47B397C70093C7F7FFE6
:10039000F98F3396C5005D8E50D982800D47338723
:1003A000E502032805019D47B397E70093C7F7FFD0
:1003B000B3F70701B396E600DD8E14C96DBFB147F0
:1003C00063E2C702954765163306F6021859FD47E2
:1003D000B397C70093C7F7FFF98F3396C5005D8EBB
:1003E00010D9828095474D163306F6025855FD47C1
:1003F000B397C70093C7F7FFF98FB395C500DD8D9D
:100400004CD582803C4993F707E0DD8D2CC9828072
:10041000376702408327074011C593E72700232051
:10042000F7408280F59BE5BF37670240832787400E
:10043000C19B5D8D2324A7408280411102C6B7670E
:10044000024003A74740137707FC3AC63247598D4D
:100450002AC6324723A2E74041018280584103283F
:1004600005004C4537060140930706403E979346EA
:10047000F8FFB1C583250640F58D2320B640D04353
:10048000F18ED4C31443B3E6060114C31841904758
:100490009346F7FF758E90C7D047F18ED4C71445A9
:1004A00041466399C6009447D98E94C7D447558F67
:1004B000D8C78280B6979443558F98C382801C43D7
:1004C000F58F1CC38280B707014023AAA740828012
:1004D0009845937707011378F70081C7DC413368AB
:1004E000F8009441814713F6F60F39C21C410146CA
:1004F000854E3D4F930F800293028004214EB398A6
:10050000CE00B3F516016391B80213132600B3159C
:100510006F0093C5F5FFED8F33136800B367F300E9
:100520006319F70F232A15010506E31AC6FD1CC13E
:100530004166130606F0758E49C637F6FF1F03267F
:1005400046701376060F7DE6371601409305068048
:100550006316B50CB707002083A70701A145854E98
:100560003D4F930F800293028004414E3393BE00AF
:1005700033F666006312C302139625000116B31802
:10058000CF0093C8F8FFB3F7F8003316C800D18F37
:100590006314F70B232A65008505E399C5FD5CC14B
:1005A00037F6FF1F032646701376060F19EA371633
:1005B0000140930506806316B508370600202328FE
:1005C000F600C16763E6F604504D8147054E3D4F86
:1005D000930F800293028004A14E93850701B31507
:1005E000BE00B3F8B6006391150393982700331348
:1005F0001F011343F3FF3376C300B318180133E62A
:10060000C800631CF7054CC98507E398D7FD50CD9A
:100610008280E31B57F02328150139B7930506C0E4
:100620006315B50083A7418015BFE319C5F283A701
:1006300081802DB75C411DB7E31057F62328650074
:10064000A1BF930506C06315B50023A2F18095BF35
:10065000E319C5F623A4F180ADB7E31757FAB31534
:10066000FE000CD155B723A4A1D4828003A781D466
:10067000854714216310F7021C31639CE7023C217B
:10068000960793E707F837E700E093F7F70F3697F9
:100690002300F740054793D756003317D70054413E
:1006A00089CE938707048A07B7E600E0B69798C318
:1006B0008280EDF33C219607F9B793870706B7E6EA
:1006C00000E08A07B69798C30F1000008280377742
:1006D00000401C43014693E727001CC3B7F700E026
:1006E00003A707D11367470023A8E7D083A707D143
:1006F000918B95C39307800873B007800F1000009B
:10070000B707014003A6474003A7074083A6474019
:10071000558F23A2E740B7F700E083A607D103A7D0
:1007200007D193F606021367870223A8E7D003A731
:1007300007D11377F7FD558F23A8E7D003A707D17B
:100740001367870023A8E7D07300501003A707D1D1
:100750001367870023A8E7D07300501083A707D141
:10076000918B89CBB707014023A2C740930780082C
:1007700073A00780828099C5371702405C4B5D8D5E
:1007800048CB8280B7170240D84B1345F5FF798DCF
:10079000C8CB828099C5371702401C4F5D8D08CFAA
:1007A0008280B7170240984F1345F5FF798D88CFA7
:1007B000828099C5371702405C4F5D8D48CF82809B
:1007C000B7170240D84F1345F5FF798DC8CF828007
:1007D00099C5371702405C475D8D48C78280B717BF
:1007E0000240D8471345F5FF798DC8C782801A218A
:1007F0008D6793870704B6217D8F9E21D58FD621E3
:10080000D58FF621D58F9625D58FB625D58FD625B0
:10081000D58FF625D58FD98F1EA19E291EA982803E
:100820001E2189C593E707041EA18280C207C183E8
:1008300093F7F7FBC207C183C5BF9386E1D48E222D
:1008400033D6A540058A0DE205473317A7004D8F23
:100850009AA2938781D613174500BA97DC4389C7BC
:10086000EFF21F8D8297FDB082809386C1D49222D1
:1008700005473317A700518F9AA2938781D6131784
:100880004500BA979C4789C7EFF29F8A8297D9B0F3
:10089000828085479386E1D4B397A700922293C7BD
:1008A000F7FFC207C1877D8E92A29386C1D49222A0
:1008B00013174500F18F9EA2938781D6BA97DC4724
:1008C00089C7EFF2FF86829771B08280EFF25F8373
:1008D000416B938481D60144014A81490149894C85
:1008E000B71B0140854A7D1B314D130C8025930DAC
:1008F000802593170401C1834DE003A58B00137578
:1009000005400DC19E20638F67018507C207C18323
:100910009EA06399A701B3978A00B3E93701C20982
:1009200093D909019A2063198701B3978A0033E9A3
:100930002701420913590901BE20D9C3938787258E
:100940006310F708B3978A0033E92701420923901F
:10095000B401135909013DC50504A947C104E31AAF
:10096000F4F80144A944B3D78940858B81C7137536
:10097000F40FE135B3578940858B81C71375F40FA8
:10098000ED35B3578A40858B81C71375F40F113746
:100990000504E31A94FC6FF06FFA63ECFC0083A784
:1009A0008BC01305A4003395AA007D8D1335150067
:1009B00089BF1305D4FF1375F50FEF00607E91B763
:1009C00041FD59DBB3978A0033EA4701420A23907D
:1009D0000400135A0A0149B775151375F50F9947A5
:1009E00063E2A704EFF2CFF48967938787890A054A
:1009F0003E951C418287A38801D4FD2A19A805478A
:100A0000A388E1D4DDBF0D47E5BF05472388E1D4C6
:100A10008D2E6FF02FF40947D5BF238801D4CDBFA9
:100A20000947F9BF8280EFF2AFF0854683A7C18006
:100A30001387C180630CD5008946630FD5000C2352
:100A4000138541E6EF00B01F6FF0CFF09146E3F859
:100A5000F6FEFD171CC3E5B785079306C002E3FB4E
:100A6000F6FE14C3E9BF37170000938781D613073A
:100A700067A2D8D398D7D8CB98CF371700001307E1
:100A8000879D9306800CB6B3B6ABD8DBF8C3F8CB22
:100A9000F8D3F8DB23A2E70823AAE7088280EFF265
:100AA0002FE983C711D505476389E7028DC309473D
:100AB000638AE7020D47638CE70283C701D50547C8
:100AC000638FE70209476386E7046FF0AFE81146DA
:100AD0008D4513050019A122CDB70946854513059B
:100AE0000032D5BF1D4691451305C05DEDB7930695
:100AF000D00F7D469305F0050D4501247DBF1307FA
:100B000000068D461306004BB94513050032C52477
:100B10006DBF8D4609469305F0031D45D52675B773
:100B200018414C4110450328C5000607B3C7C5004E
:100B300005833D8F9316170093571800B98EB3C7DE
:100B40000701B58F1397A700358F5CC50CC150C145
:100B500018C5858B99C71C49B18F5CC15C493D8F15
:100B600018C58280EFF2CFDCB717708F9387E71E2E
:100B70001CC95CC1B70779FC9387F7F15CC91CC538
:100B8000B70794379387F7DF3796076C2A840CC131
:100B90001CCD5CC505472145130656966319A70071
:100BA000A1442285FD14AD3FEDFC6FF0AFDA930751
:100BB000F7FF8D8B8A07A2978C43937637008A06BE
:100BC00093D7E501AD8FB387C702A2968C42BA973F
:100BD000AD8F9CC20507D9B7EFF28FD52A8489372C
:100BE0001C4418404844A183BA973D8D858B99C316
:100BF0001C4C3D8D6FF00FD6938741E223A0070078
:100C000023A2070023A4070023A6070023A80700A8
:100C100023AA070023AC070023AE07008280130736
:100C20000008930700F86363C700B28713F6F70F55
:100C30001387C1EB1388C1EB9386C1EB13038705C0
:100C40009307F00C930800FD034E080063F4C701FE
:100C5000230018010508E31903FF938741E283A8E5
:100C60000700638908020548638008059306F006BB
:100C70001C2363F4F600918F1CA31C2363ECC706AE
:100C8000918F1CA30507E315E3FEEFF26FCA7926E7
:100C90006FF04FCCD44391E6054798C323A40700D7
:100CA0008280FD16D4C3D9B703A84700631C08028D
:100CB000CCC38C471388150023A4070113087005C3
:100CC0006366B802B387B6009306000294A3D9DD29
:100CD00093066006A38FD7FEE38A15F9BD56238FCE
:100CE000D7FE69B77D1823A2070149B723A00700E3
:100CF000C8C3ADBFC1DBFD1769B7EFF26FC0138783
:100D000041E25C438507AA8D2E89B28AB68C5CC30A
:100D1000014D138441E24E8B9384C1EBAA8B0D4CA1
:100D2000130A8005138581E0453D1375F50F63793E
:100D30005501B3069D009C2263FBFD0285839CA2A6
:100D4000636195035C408D8B89EF138581E0693584
:100D500033079D001C233E951375F50F6360A902B0
:100D600008A3050DE3104DFD552C6FF02FBD5E87D8
:100D70006373BC010D477D17BA97D1B723002701D4
:100D8000CDB7EFF2EFBA938741E423A0070023A287
:100D9000070023A4070023A6070023A8070023AA0F
:100DA000070023AC070023AE07001387C1EB9306AF
:100DB00047019387C1EB230C07040507E31DD7FE0A
:100DC00023860706A3880706A38607062389070646
:100DD00023870706A3890706A3870706238A070632
:100DE00023880706A38A0706152C6FF0AFB6854740
:100DF0006393F6008946138841E48328080005437D
:100E0000938741E463876804638A0802094763871C
:100E1000E8020D47638CE80AEFF28FB19387C1EBCC
:100E20009386570003C7470685072388E706A385EF
:100E3000E706E399F6FEDD226FF0CFB1D84319E75C
:100E4000850823A0170123A4070082807D17D8C33B
:100E5000E1B783274800B9EB032588002322B800B7
:100E6000930715002324F800A94763E5A704138816
:100E7000C1EB1386C1EB9387C1EB83C51706B6950B
:100E800093F5F50F636EB702A380B7068345160688
:100E9000B69593F5F50F6368B702A300B6067D1605
:100EA000B305C8408507E37AB5FCBDB7FD1723221B
:100EB000F8009DB789472320F8002322C80045BFCA
:100EC000A380E706E1B7A300E606D1BF85821387BA
:100ED000C1EB94C793084701814503468705014844
:100EE0006366D600158E1378F60F8505230C07056B
:100EF0000507E394E8FE8DF123A00700C8C329BFCE
:100F0000138741E45843938741E431E3984B21E749
:100F1000D847C8C349480507D8C76367E804C84726
:100F200098432A8801C749483308A8401387C1EB72
:100F30003A98230CB8040948637BA8001D48636EE7
:100F4000A8023305A8402A9785812306B706D8430F
:100F50007D17D8C321A07D1798CB5DDB98471DC7AF
:100F600098477D1798C7828098430A0523A60700F3
:100F70001347170098C388CB5DB74D151148E36838
:100F8000A8FC2A978581A308B706D1B71387C1EBC0
:100F900090C71305E70103468705814563F5C60041
:100FA000158E9375F60F230CB7040507E315A7FEFE
:100FB00045BFEFF2EF97B71701401307000823A8CA
:100FC000E7C04111B70702003EC6B2471387F7FFDB
:100FD0003AC6E5FF938441E71306800481451385F3
:100FE00041E7EFF0EF97938741E64147B146194655
:100FF000138541E69305600784C78126D145138593
:1010000041E63529138541E6C9261306700481455A
:10101000138541E6C92141016FF0CF93054723892C
:10102000E1D48280938721D5982321CBEFF24F9092
:101030008966238007009386468B81479308700456
:10104000138641E79385C1EB130860073387F600E9
:1010500018231305F7FF1375F50F63E8A800338510
:10106000F50008213297A30FA7FE8507E39007FF3D
:10107000138541E6992E6FF0EF8D8280EFF24F8B52
:1010800079711306000281450808EFF06F8D938691
:1010900041F305671386060C938741F3130810F894
:1010A0001305C00493050780A3800601A8A2EEA241
:1010B000E106E39BC6FE930540052385B7041306AE
:1010C000C7DF9305A7D79306F004B4A3F2AF930646
:1010D00047D32397B704094693054004F6A3238812
:1010E000C702F6BB2381B706239FD706930587BBAC
:1010F0001306F006B5461307E7DD372401402389C0
:10110000C7022393B7060D462388D708239BE70819
:101110009306A0041307902005499144A145238913
:10112000D7082394E70A2384C7042385C70A238C9E
:10113000270123809706238CB70623800700130519
:101140000440EFF02F951305044093055002EFF093
:101150006FABB7070E000C08130504403ECE230208
:10116000210302C802CA02CC02D0EFF0EF941305AB
:1011700004408545EFF0AF99F5477C8405468547E7
:1011800093050022130504403EC64485EFF02F99D5
:10119000280023200440EFF06FCD45616FE09FFBF6
:1011A00085473395A70083A741D57D8D3335A000B2
:1011B0008280B72701401387074083A70740898BA8
:1011C000A1CB03C631D5E145B146B305B6021385BF
:1011D00041F30328C704938741F3B306D602AA95C7
:1011E000B831BA968606AA962394060194318545AD
:1011F00093F6F6076383B6020D48A14505071377FA
:10120000F70F637FB700E1463306D602B297B8B353
:10121000B727014023A00740828009489145F9BFC4
:1012200061473307E602014581463E97A301070067
:101230008358870005050907C696E34BB5FE61474D
:101240003307E602B3D60601139506014181BA972A
:10125000CAA31147E39EE5FAFA23636AA7009385C0
:1012600041D588418547B397C700C98F9CC1C20645
:10127000C18213072704E35DD7F8138741D51443D0
:101280008547B397C70093C7F7FFF58F1CC349B7CE
:10129000EFE21FEA9D89411193E505FC2AC6238AE6
:1012A000B1FE97F0FF1FE78000E732458145082136
:1012B00097F0FF1FE78020291305000F97F0FF1F0D
:1012C000E780C0158545138541FF192E97F0FF1F54
:1012D000E78000F741016FE0FFE7EFE27FE53C21A7
:1012E0002A84AE849D8B91C781455D373C20E19B6C
:1012F0003CA0B3379000238AF1FE97F0FF1FE780F0
:1013000080E10820814597F0FF1FE780C023054555
:1013100097F0FF1FE78080108545138541FFC924A2
:1013200097F0FF1FE780C0F138209377F70799C047
:10133000936707083CA06FE0FFE1EFE2DFDD937900
:10134000070F411154A10CA130B1A3003501814513
:101350002A8432C659373246138941FF7D1623004D
:10136000C90097F0FF1FE78000DB0820814597F058
:10137000FF1FE780401D1305000897F0FF1FE7805F
:10138000E009138541FF8545A12C97F0FF1FE780F9
:1013900020EB2300390197F0FF1FE780C0D708201A
:1013A000814597F0FF1FE780001A0D4597F0FF1F5A
:1013B000E780C0068545138541FF1D2497F0FF1F78
:1013C000E78000E841016FE05FD8EFE2DFD43C2125
:1013D00009472A849D8B6389E7008945553D3C2058
:1013E000E19B93E727003CA001498144314AB3893E
:1013F00044033C3093F9F90F63E4F4006FE0FFD449
:1014000097F0FF1FE78020D108208145850497F0E1
:10141000FF1FE78040134E8597F0FF1FE780000015
:1014200008444C2093F4F40F4A955D2A97F0FF1F6F
:10143000E78000E15C203E991379F90F4DBFEFE2A0
:101440009FCD1307F0032A849307F0036363B7006B
:10145000AE8793F4F70F3C2005479D8B638AE70026
:101460008545228535353C20E19B93E717003CA05C
:101470008147938641FFBA893387F60004A3582039
:10148000850793F7F70FE379F7FE8144314A3389F3
:1014900044033C301379F90F63E4F4006FE0FFCAB2
:1014A00097F0FF1FE78020C708208145850497F04B
:1014B000FF1FE78040094A8597F0FF1FE78000F68D
:1014C0004C20138541FF93F4F40F192A97F0FF1F66
:1014D000E78000D76DBFEFE21FC43C214111AA8411
:1014E0009D8BAE8981CB814532C65D33BC203246AF
:1014F000E19BBCA00147B148138341FF194E854EC3
:10150000314FB3071703B4301314170093F7F70FD5
:10151000636FD70297F0FF1FE780E0BF8820814507
:1015200097F0FF1FE78020021305100397F0FF1FBD
:10153000E780C0EE93150401C181138541FF4D2062
:1015400097F0FF1FE780C0CF41016FE01FC0B305D8
:101550008300A3800500238005008146014563CAFE
:101560003703634CF60283CF440013F8F60F63721F
:10157000F8036316C80119051375F50F850583CFA8
:1015800005003388A64033980E013368F8012380A4
:10159000050185068507E394E6FD05071377F70F38
:1015A0008DB7B717014003A747C0419B136747009A
:1015B00023A2E7C01307001023AAE7C003A747C070
:1015C0001377F7F01367070423A2E7C0130700207F
:1015D00023AAE7C00547239CE1D4239D01D4828040
:1015E000EFE21FB5AA95939405012A84C180931751
:1015F0000401C183638AF40005040345F4FF97F0F6
:10160000FF1FE780A0E165D56FE0DFB4EFE25FB2D6
:10161000011102C69307401002C87C878947FC81EC
:10162000B707000285076C00373501403ECA02CC7F
:10163000231E0100EFF0AF9B854537350140EFF0E9
:101640002F9E05616FE01FB101A041113EC4B70795
:10165000EFBE3AC69387070837E700E03CC701A012
:10166000893E73002030EFE2BFAC01110545EFE089
:101670009FFF6122056585451305D521EFF08F9108
:10168000854537050010EFF0CF92370502008545FC
:101690000505EFF04F8E371401408544FD471305D3
:1016A00004800C083EC802CC26CAEFE07FE2130596
:1016B00004C00C0826C8EFE0BFE1A5470C083715A9
:1016C00001403EC8EFE0DFE0E147130504803ECC77
:1016D0000C089307000A3EC8EFE09FDF93078004E1
:1016E000130504803ECC0C08930700043EC8EFE0CD
:1016F0003FDE8967938787B0130504C00C083EC896
:10170000EFE01FDD93078002371501403ECC0C0847
:10171000B70703003EC8EFE0BFDB9307004F130598
:1017200004C05CC941470C083ACC3EC8EFE05FDA20
:10173000EFF08FCCBD35EFF0DF87EFF03F94F93558
:10174000EFF06FB293059053138581E0EFF08FC1F6
:10175000014502C802CA02CC02CEEFE0FFCC13055D
:10176000F002EFE09FCD0545EFE09FCAB707000804
:101770003EC80808A1473ECC02CA26CEEFE01FCEE5
:10178000D54728007C842305010026C6EFE01FEE24
:10179000138701D61C2393F7F70F89C7230007008F
:1017A000EFF0EFAFEFE0BFF2E5B737050008EFE08D
:1017B0009FD11387E1D51E239306703E8507C2078C
:1017C000C1831EA363FDF600938741D62310070053
:1017D0009843050798C305472380E1D629A02947E8
:1017E000B3F7E702EDDBEFF0FF8397F0FF1FE78031
:1017F000E083EFF0AF8D73002030B7160240DC427B
:10180000918313F7F700B707002093870700BA9773
:101810009C23D4423777DC0293F7F70F130707C0F6
:1018200093F606083356F70099E23356F70223A8D9
:10183000C1808280372702401C43F19B93E627003A
:1018400014C337170240544393F6F6F054C354437D
:10185000C98E54C309C941476314E50093E71700D3
:10186000372702401CC38280EFE29F8CB7170240EB
:101870009843B70600F99386F6F51367170098C3E7
:10188000D843414513670705D8C3D843758FD8C3DC
:1018900055376FE03F8C0000F6090000FE0900009C
:1018A000060A00000A0A0000160A00001A0A0000D0
:1018B000200A00000D190131250E1A022632031BE1
:1018C0000F273304101C283405111D293506121E5C
:1018D0002A36000000000000070013001F002B0044
:1018E00037000000000000000000000000000000C1
:1018F00000000000000000000000000000000000E8
:10190000000008000014000020000000091521005C
:1019100000002D390A16222E3A0B17232F3B0C00FC
:0C192000434647482C3C30241838000097
:10192C000102030405060708010203040506070863
:10193C004444444444444444444444441400000057
:10194C00006CDC0200000000E7020013411183C7A9
:10195C0031D5A3070100138631D5138741F3E14834
:10196C001D4885079D8BB3861703BA9694329395C1
:10197C008601E18563CC05008C8793F5F50F138503
:10198C0015001375F50FC887E37DB8FC1CA2908772
:10199C00A1456385C50293F6F6F705466383C60237
:1019AC000946638CC60499EAB727014003A7474050
:1019BC00B70600FFFD16758F23A2E74041016700B3
:1019CC004015E144B38797023724014083264440F5
:1019DC003706000113040440D18E54C005469D46C1
:1019EC002285B304F7008C20E700C034BC2013F729
:1019FC00070F58DCBD8B7CC4D1B73724014083263C
:101A0C004440370600FF7D16F18E2322D440E14678
:101A1C00B387D7021304044022850546BA97B42332
:101A2C008C23BD8AE700C03485452285E70040330E
:101A3C0071B737170140832747C093F7F7F093E747
:101A4C0007042322F7C003D681D51387C1D512A36F
:101A5C009387C1D59A23420741839306F7FFC206A9
:101A6C00C18296A365FBB716014003A746C0419BF4
:101A7C001367470023A2E6C092A39A23420741832F
:101A8C009306F7FFC206C18296A365FB3716014089
:101A9C00032786C01377071065DF032746C013772B
:101AAC00F7F0136707012322E6C003D6A1D592A352
:101ABC009A23420741839306F7FFC206C18296A37D
:101ACC0065FBB716014003A746C0419B136717007F
:101ADC0023A2E6C092A39A23420741839306F7FF01
:101AEC00C206C18296A365FB8280E70200133717FA
:101AFC000140832747C093F7F7F093E707042322AD
:101B0C00F7C003D681D51387C1D512A39387C1D54E
:101B1C009A23420741839306F7FFC206C18296A31C
:101B2C0065FBB716014003A746C0419B13674700EE
:101B3C0023A2E6C0B716014003A786C0137707108F
:101B4C0065DF92A39A23420741839306F7FFC206EF
:101B5C00C18296A365FBF13D670040153717014024
:101B6C00832747C093F7F7F093E707012322F7C0C9
:101B7C0083D6A1D51387C1D516A39387C1D59A2334
:101B8C00420741839306F7FFC206C18296A365FB09
:101B9C00B716014003A746C0419B1367470023A219
:101BAC00E6C003D781D59AA39623C206C1821386B9
:101BBC00F6FF4206418292A3E5FAB715014083A6CF
:101BCC0085C093F60610E5DE83A645C093F6F6F0C5
:101BDC0093E6060423A2D5C09AA39623C206C1821B
:101BEC001386F6FF4206418292A3E5FA9AA3962346
:101BFC00C206C1821386F6FF4206418292A3E5FA21
:101C0C009AA39623C206C1821386F6FF420641822E
:101C1C0092A3E5FA9AA39A23420741839306F7FF0E
:101C2C00C206C18296A365FB8280371701408327C9
:101C3C0047C0A146B718014093F7F7F093E70704A4
:101C4C002322F7C003D881D583D5A1D5014783A71B
:101C5C0048C006071377F70FC19B93E7470023A2F1
:101C6C00F8C083A788C093F70710E5DF9387C1D529
:101C7C00239007019223420641821303F6FF42038D
:101C8C00135303012390670075F6138308C00326D2
:101C9C0083001376062019C213671700032643002E
:101CAC00419A136616002322C3008EA39223420688
:101CBC0041821303F6FF4203135303012390670081
:101CCC0075F6FD1693F6F60FD9F2B716014093860A
:101CDC0006C0D0421376F6F029CD13660601D0C2A9
:101CEC0037160140832646C0C19A93E6460023224C
:101CFC00D6C0239007019623C206C1821386F6FF35
:101D0C004206418292A3E5FA37160140832646C06B
:101D1C00C19A93E616002322D6C08EA39623C20640
:101D2C00C1821386F6FF4206418292A3E5FA3A85F8
:101D3C0082801366060465B737170140832747C0B6
:101D4C00C19B93E717002322F7C003DE81D583DE06
:101D5C00A1D52147938581D51386A1D5371801408C
:101D6C0093178501E187930608C063D6070EDC4202
:101D7C0093F7F7F093E70704DCC2832748C0C19BB5
:101D8C0093E747002322F8C0832788C093F70710F6
:101D9C00E5DF9387C1D52390C7019623C206C18284
:101DAC009388F6FFC20893D8080123901701F5F623
:101DBC00832648C006051375F50FC19A93E61600E5
:101DCC002322D8C02390D7019623C206C1829388C0
:101DDC00F6FFC20893D8080123901701F5F67D177A
:101DEC001377F70F35FF37170140130707C054431C
:101DFC0093F6F6F093E6060454C301005443C19ADB
:101E0C0093E6460054C39A219AA39A23420741832E
:101E1C009306F7FFC206C18296A365FBB715014076
:101E2C0003A785C01377071065DF03A785C003A739
:101E3C0045C0419B1367170023A2E5C01A229AA341
:101E4C009A23420741839306F7FFC206C18296A3E9
:101E5C0065FB01458280DC4293F7F7F093E70701BD
:101E6C0021BFE7020013B335B0001375E50F4D8D9C
:081E7C00E1356700401500008C
:00000001FF
